:0A000000D7C064C1E0C1FCCFEEC11F
:10000A00FACFF9CFF8CFA4C190C1F5CFF4CFF3CF8F
:10001A00F2CFF1CFF0CFEFCFEECFEDCF3E4141415E
:10002A003E00007F02040000464951614200364901
:10003A00494122007F080808070031494949270039
:10004A00324949493E00030D7101010036494949C7
:10005A0036003E49494926000014400000003E414E
:10006A0041413E000010207F0000214345493100F4
:10007A00224149493600700808087F0072494949F7
:10008A0046003E49494926004040475860003649E3
:10009A0049493600324949493E000014010000002E
:1000AA007C0A090A7C00364949497F00414141419D
:1000BA003E003E4141417F00414149497F000101E3
:1000CA0009097F00324949413E007F0808087F003C
:1000DA0000007F000000003F404020004122140839
:1000EA007F00404040407F007F0204027F007F1073
:1000FA0008047F003E4141413E00060909097F008C
:10010A003E6151413E00661909097F003249494959
:10011A00260001017F0101003F4040403F001F20AF
:10012A0040201F007F2010207F0063140814630002
:10013A0007087008070043454951610018FC18FC7C
:10014A00060005000400030002000100030001008C
:10015A00010005000D0002000B00460102000D001F
:10016A004801010061014A01010062014C010100DC
:10017A0063014E0101006401500101006501520151
:10018A00010066015401010067015601010069017D
:10019A00580101006A015A0101006B015C0101006A
:1001AA0084015E010000F894EE27ECBBF1E0FBBF8E
:1001BA00EBBFE5BFF8E1F1BDE1BD8DE0A2E0BB27F1
:1001CA00ED938A95E9F780E094E0A0E6ED93019734
:1001DA00E9F7E0E6F1E085919591009761F0A59144
:1001EA00B59105901590BF01F00105900D92019708
:1001FA00E1F7FB01F0CFEFE5EDBFE4E0EEBFC0E6CB
:10020A00D1E022C3E881EF73E064E5BBE881E074E2
:10021A00E295EF70E695E695EC60E2BB21960895CB
:10022A004ED50B2D1C2DA02FB12FE0E1F7E234D5CE
:10023A00E0936801A0E1B7E255D40E1B1F0BA02F73
:10024A00B12FE8EEF3E028D5E0936701A8EEB3E01A
:10025A0049D40E1B1F0BA02FB12FE4E6F0E01CD5EA
:10026A00E0936A01F0E02E2F3F2FE22FF32FA4E64E
:10027A00B0E00AD50E1B1F0BA02FB12FEAE0F0E069
:10028A000BD5E0936901F0E04E2F5F2FE42FF52F95
:10029A00AAE0B0E0F9D40E1B1F0BE02FF12FE09378
:1002AA006C0114D52696089520D423D426D429D4B3
:1002BA002CD42FD432D435D438D43BD43ED441D4E0
:1002CA0008950A921A929A93AA93BA93EA93FA937E
:1002DA00EFB7EA933AD4919ACDBCBCBC7724882470
:1002EA00E0916E01EF5FE0936E01E37069F4E92D2E
:1002FA00FA2DC5D4DF01E7E2F0E0CED4A9EFBFEFD3
:10030A00AE1BBF0BBA2ECB2E9924AA2421D4E89473
:10031A0023F8689420F8E991EFBFF991E991B9912E
:10032A00A991999119900990189515D40A9302B731
:10033A00E02FE053E2BF919A689421F8E1E0F0E0FF
:10034A004E0E5F1E9E0EAF1E9198099109D4189504
:10035A0002D4B9D40CB51DB5E02FF12FEB0DFC1D5D
:10036A003796FDBDECBD689422F8E1E0F0E07E0E20
:10037A008F1EE5EEF1E0E715F80529F4E1EEF1E06C
:10038A007E2E8F2E23F8E6E0E61509F4E1D3A5D4F4
:10039A00E7D31895EAD3E5B7E37FE5BFE5B7E860A9
:1003AA00E5BFE0E8EABFE5D3E89426F8E5D3E0E064
:1003BA00E0937C01E0937D0178940895EA93EFB786
:1003CA00EA93DED3E9B7E064E9BF26FE03C0EBB7E0
:1003DA00EF77EBBFE991EFBFE9911895AA93BA932A
:1003EA00EA93FA93EFB7EA93CBD3CDD369F0E091CE
:1003FA008301E150E0938301C6D329F4E9B7EF7B87
:10040A00E9BFC5D3B2D36BC0A0918201E1E0EA177C
:10041A0058F4689426F8BBD3839B02C0BCD302C0AD
:10042A00E5B7E460E5BFA1D3E0918201E03061F471
:10043A00E0E0E0938001E0938101E0E0F0E8E093FE
:10044A007E01F0937F0115C0839B13C0A0918201A6
:10045A00E2E0EA1770F4E0917E01F0917F01A09149
:10046A008001B0918101EA2BFB2BE0938001F0938C
:10047A008101E0917E01F0917F01F695E795E09385
:10048A007E01F0937F01A0917E01B0917F01A03897
:10049A00E0E0BE0731F4E0E2F0E0E0937E01F093A1
:1004AA007F01A0918201AF5FA0938201A150AF307A
:1004BA00B1F46DD370D3E5BFE0E0E0938201E89434
:1004CA0026F8E0918001F0918101E0937C01F0939C
:1004DA007D01E1E0E0937B01E0E9E0938301E991AA
:1004EA00EFBFF991E991B991A9911895E09161014C
:1004FA00EF5FE0936101A091610150D308F043C01E
:10050A00E0E0E0936101E0916201EF5FE093620154
:10051A00A091620146D3B8F5E0E0E0936201E09170
:10052A006301EF5FE0936301A091630137D358F54C
:10053A00E0E0E0936301E0916401EF5FE09364011E
:10054A00A09164012ED3F8F4E0E0E0936401E09115
:10055A006501EF5FE093650127D321F4A09165015E
:10056A00A43009F006C024D3E0E0E09366010CD081
:10057A000AC0A091650112D330F41AD3E091660142
:10058A00EF5FE09366010895A0916701A83061F4D6
:10059A00A0916801A23041F4A0916901A23021F42E
:1005AA00A0916A01A03009F004C006D3E3E0E09309
:1005BA006901A0916701A03011F404D309F01BC0AE
:1005CA00E0916901E43011F0E63019F4F5D2FED277
:1005DA0012C0E93041F4F0D2E0E0E0936901E1E0D1
:1005EA00E0936A0108C0E13031F4F6D221F0E4D296
:1005FA00E2E0E0936901A0916701A13011F4E2D22F
:10060A0009F029C0E0916901E13029F4E5D211F439
:10061A00D3D2DCD220C0E33011F0E53009F402C0B5
:10062A00E73009F402C0E83009F402C0E03019F4F6
:10063A00C3D2CCD210C0E23071F4CED261F0BCD2B7
:10064A00E1E0E0936901E0E0E0936A01E0916B0187
:10065A00EF5FE0936B01E0916701EF5FE093670161
:10066A00A0916701AA3041F4E0E0E0936701E091CC
:10067A006801EF5FE093680108950A937DD2E091E3
:10068A007D01E53009F0DEC0E0918401EF5FE0937F
:10069A00840100E0E0917C01E03221F405DEE0E033
:1006AA009FD24CC0E13221F4FFDDE6E099D246C088
:1006BA00E63329F4F9DDEDE0E09384013FC0E43349
:1006CA0019F4E0E12E263AC0E23359F48ED291D2DF
:1006DA00E9E0E093630191D294D2E7E0E09361010B
:1006EA002DC0E13019F401E0A99A28C0E23019F4CA
:1006FA0002E0AA9A23C0E33019F403E0AB9A1EC0C1
:10070A00E43019F404E0AC9A19C0E53019F405E0B4
:10071A00AD9A14C0E63019F406E0AE9A0FC0E7307D
:10072A0011F407E00BC0E83011F408E007C0E93023
:10073A0011F409E003C0E03009F400E0E09184011B
:10074A00E03021F4EAEFE0936F017CC0E13059F424
:10075A00CCD1EAEFE0937001033018F400936601FC
:10076A0001C047D26FC0E23079F4C3D1EAEFE09317
:10077A0071011AD219F4E3E0E01708F002C035D289
:10078A0002C0009365015EC0E33059F4B6D1EAEFC6
:10079A00E0937201063018F40093640101C02DD26F
:1007AA0051C0E43039F4ADD1EAEFE093730100931C
:1007BA00630148C0E53059F4A8D1EAEFE093740127
:1007CA00063018F40093620101C01BD23BC0E63028
:1007DA0039F49FD1E9EFE0937A010093610132C0C5
:1007EA00E73039F4AED1E9EFE0937901009368017B
:1007FA0029C0E83039F4A1D1E9EFE09378010093F8
:10080A00670120C0E93039F494D1E9EFE093770128
:10081A0000936A0117C0EA3039F487D1E9EFE0930F
:10082A007601009369010EC0EB3039F47AD1E9EF11
:10083A00E093750100936C0105C0EC3019F46DD199
:10084A0000936B0109910895E0E0E8BBEFE3E7BB91
:10085A00E0E4E5BBEFE7E4BBECE0E2BBE1E0E1BBEF
:10086A00E2E0E3BFE0EEE2BFE0E0EFBDE2E0EEBDD2
:10087A00ECEFEDBDE8E1ECBDE0E0EBBDEABDE9BDC2
:10088A00E8BDE2BD76D1E0E0E4BDE3BDEBB7E06CE4
:10089A00EBBFEAE0E5BFE0ECEABFE5E4E9BFE0E888
:1008AA00E8B9E0E0E0BFEFE1E1BDEFE0E1BD789457
:1008BA0071DDFADC689425F820FE04C0E89420F87B
:1008CA0024FCAEDC22FE31C0E89422F89ED139F530
:1008DA0025FE1BC0A6E2B0E0E0916D01F0E0BF93F7
:1008EA00AF93A2E4B0E0D0D1AF91BF91AE0FBF1FDA
:1008FA0090D1BF93AF9391D1AF91BF9192D1A09173
:10090A006001AA3008F463940AC0AAEAB0E081D16F
:10091A00BF93AF9382D1AF91BF9183D1639475D1C5
:10092A00E23019F4E0E0EA936DDC21FE0DC0E894B0
:10093A0021F8E2ECF2EAE415F50530F444245524F2
:10094A00D5DD23FC909AA895E72DF82DE330A0E099
:10095A00FA0739F4E09178016DD1E0916A016FD11B
:10096A00BAC0EB31A0E0FA0721F46DD16ED171D192
:10097A00B2C0EF31A0E0FA0711F46ED1ACC0E33295
:10098A00A0E0FA0739F4E091790154D1E0916701C6
:10099A0056D1A1C0EB33A0E0FA0739F4E0917A010D
:1009AA0049D1E09168014BD196C0E73AA0E0FA0735
:1009BA0039F4E0916F0155D1E091660140D18BC0C5
:1009CA00EF3BA0E0FA0739F4E09170014AD1E091D7
:1009DA00650135D180C0E73DA0E0FA0729F4B5D01A
:1009EA0045D133D147D177C0EB3DA0E0FA0719F4DE
:1009FA003DD143D170C0EF3DA0E0FA0739F4E09150
:100A0A0071012FD1E09164011AD165C0E73FA0E0DE
:100A1A00FA0739F4E091720124D1E09163010FD110
:100A2A005AC0EF30A1E0FA0729F48FD01FD10DD1B7
:100A3A0021D151C0E331A1E0FA0719F417D11DD130
:100A4A004AC0E731A1E0FA0739F4E091730109D10C
:100A5A00E0916201F4D03FC0EF32A1E0FA0739F425
:100A6A00E0917401FED0E0916101E9D034C0EF3821
:100A7A00A1E0FA0739F4E0917501DCD0E0916B014D
:100A8A00DED029C0E73AA1E0FA0739F4E09176010D
:100A9A00D1D0E0916C01D3D01EC0EF3BA1E0FA07A0
:100AAA0021F4D1D0D2D0D5D016C0E33CA1E0FA07C8
:100ABA0011F4D2D010C0E73CA1E0FA0739F4E09172
:100ACA007701B8D0E0916901BAD005C0EF3DA1E045
:100ADA00FA0709F4C1D0E0917B01E03009F0CDDDDD
:100AEA00EBCEFFCFF0E0D0D00895E9EFE0936F01AD
:100AFA000895E9EFE09370010895E9EFE093710139
:100B0A000895E9EFE09372010895E9EFE093730124
:100B1A000895E9EFE09374010895EAEFE09375010F
:100B2A000895EAEFE09376010895EAEFE0937701FA
:100B3A000895EAEFE09378010895EAEFE0937901E6
:100B4A000895EAEFE0937A010895EAEFE8BB089581
:100B5A00E5E06E2E0895EA93FA93EFB7EA930895C3
:100B6A00E991EFBFF991E9910895EBB7E068EBBF1E
:100B7A000895E6E0E5BD0895E0E0E0937B0108957D
:100B8A00EEEAE4BD0895E0918301E0300895EAB702
:100B9A00EF77EABF0895E5B7EB7F0895E9E0EA1732
:100BAA000895E5E0EA170895A0916601A230089534
:100BBA00E0E0E09365010895E0E0E0936701E093E7
:100BCA0068010895A0916801A3300895E091690130
:100BDA00EF5FE09369010895E0916A01E0300895BA
:100BEA00E0938401EFEFE5BB0895E3E0E09365014C
:100BFA000895E2E0E09366010895E5E0E093640178
:100C0A000895E5E0E09362010895E72DF82DE37079
:100C1A000895E0916001F0E00895A6E0B0E034D0D4
:100C2A000895AE0FBF1FE62DF0E0EA0FFB1FE49117
:100C3A00EA93E8CAE8BBE0E0E0936D010895E09327
:100C4A00600166240895E9EFF5CFEAE0E0936001D8
:100C5A000895E2E06E2E0895E0E0E0936D01EAE087
:100C6A00EECFE8BBE1E0E0936D010895E1E0E093A7
:100C7A006D010895E1E06E2E0895EAE0E0CFEE0FEF
:100C8A00FF1FEE0FFF1F0895FA9FF02DEB9FF00D47
:100C9A00EA9FE02DF10D08950024112490E1AA0F96
:100CAA00BB1F001C111C0E1A1F0A18F40E0E1F1E61
:100CBA0001C0A1609A9599F7FD01D00108955A9350
:100CCA004A933A932A931A930A9308955D814C8121
:100CDA003B812A8119810881089509911991089502
:00000001FF
